:1000000000100020A5020000AD020000AF020000B9
:10001000B1020000B3020000B5020000E6DFFFDF1E
:10002000000000000000000000000000B702000017
:10003000B902000000000000BB020000BD02000089
:10004000BF02000079030000BF020000BF020000F1
:10005000BF020000BF020000BF020000BF0200009C
:10006000BF020000BF020000BF020000BF0200008C
:10007000BF02000000000000BF020000BF0200003D
:10008000BF020000BF020000BF020000BF0200006C
:10009000BF020000BF020000BF020000BF0200005C
:1000A000CF2C0000BF020000BF020000BF02000012
:1000B000BF020000BF020000BF020000BF0200003C
:1000C000BF020000BF020000BF020000BF0200002C
:1000D000BF020000BF020000BF020000BF0200001C
:1000E000BF020000DFF80CD005F096F8004800478A
:1000F0009F07000000100020D0F800D0D0F804F0D6
:1001000070B50023084D0AE0CE5C04885B1C86EACB
:1001100014269BB235F8166086EA04240480521E29
:1001200092B2F1D270BD00002C56000030B4554C94
:10013000534A0323C4F8B031136843F48033136087
:10014000514A30BC104710B572B633244F4B10C320
:1001500007C34F484FF47A710068B0FBF1F01860A4
:10016000191D4A48FFF7E2FF62B610BD474A322325
:100170001360C2E9010146484FF47A710068B0FB90
:10018000F1F0D06002F114011046CFE73F4A34236A
:100190001360C2E901013E484FF47A710068B0FB78
:1001A000F1F0D06002F114011046BFE710B572B64D
:1001B0000624384951F82420824212D93549783929
:1001C00051F82410814207D121460846FFF7CEFF9F
:1001D00021460846FFF7DAFF21460846FFF7C6FF2B
:1001E00002E0641C1D2CE5D962B610BD2DE9F0417A
:1001F000294C236803B92060244D0020283563680A
:1002000003E00F5C1E18401CAF559042F9D39818BC
:100210004FF480766060B04213D12068FFF7C6FFCC
:100220001A4D1435286800B1FEE7184932462831C6
:100230002068FFF788FF286800B1FEE700206060B3
:1002400020600020BDE8F08172B61449144A0140D4
:100250001160FFF751BF46F2044000210088A0F56D
:100260001942993A0AD04FF4C0404FF4002208C80E
:1002700090421944FBD309B1002070470120704718
:1002800088C10F4000C00F40F11FFF1F1C1C001051
:10029000E8000010E4590000C400001080FFFF1FB8
:1002A00008ED00E00648804706480047FEE7FEE705
:1002B000FEE7FEE7FEE7FEE7FEE7FEE7FEE7FEE716
:1002C000871A0000E500000010B50B4604461146F1
:1002D000184604F08DFFC4E9000110BD02E008C813
:1002E000121F08C1002AFAD170477047002001E0B0
:1002F00001C1121F002AFBD170470000FFFFFFFF62
:10030000EFF3108010F0010F72B64FF080404FF005
:10031000000202704FF0AA0202724FF055030372FE
:100320004FF0FF0444604FF0030404700272037244
:1003300000D162B6FEE770B500251024032001F05D
:100340001DFCC0F30B100544641EF7D129094FF4BE
:100350007A70B1FBF0F06422B1FBF2F100070A22DF
:10036000B1FBF2F302FB131141EA1060014908608E
:1003700070BD0000DC00001010B54FF040210120DE
:10038000086001F0C2FA01F04AFC10BD4FF04020B5
:100390000021016702224260C1600321416147F2EE
:1003A000305181610B4B182183F8001401215B1E31
:1003B000C3F80021416000207047074802214160D6
:1003C0000021016741611D22C260C16301214160BA
:1003D0000020704701E000E00000094040EA01030E
:1003E0009B0703D009E008C9121F08C0042AFAD2EB
:1003F00003E011F8013B00F8013B521EF9D27047AF
:10040000000000004D0B000010B5FE494869800453
:100410000CD4FD4A906843F698239468241A9C42B1
:10042000FBD34869800401D4012010BD052000F0F1
:10043000E5FF002010BD70B5F34CA668042000F065
:10044000DDFFF24D03E000BFFFF7DEFF48B1A0681B
:10045000801BA842F8D308E0FFF7D6FF08B10120BF
:1004600070BDA068801BA842F6D3002070BD2DE9A6
:10047000F041092000F0C2FFE54800264FF47A77EA
:100480000670C821384601F020FADF4CA06842F21D
:100490001075A168091AA942FBD3C821384601F09A
:1004A00014FAA068A168091AA942FBD3C8213846EA
:1004B00001F00BFAD748022186708171C670BDE841
:1004C000F0818AB04FF0000946208DF814008DF8B5
:1004D00017904520CA4600905446CFA3CFA20A21C8
:1004E00005A804F0C9FECF4908684FF6FF02104086
:1004F000CD4A40F4807010430860CC48CD49D04DBF
:100500000460CB480068A0F56C50FF380860CA4909
:1005100000F5E0500860C949400A0860F8202870DA
:10052000FF206870A87001F06BF9BA4CC54A002032
:1005300094F9051052F821102A1802F580520B5C2C
:10054000401C82F800386028F6D34FF4E175294644
:1005500040F2491001F0B9F9294640F29F1001F02C
:10056000B4F94FF4005BDFF8E0825D46207808B113
:1005700002F02EFCA07928B1012818D0207800289C
:1005800079D0FCE00A2000F039FF00F01FFE10B126
:10059000FFF76DFFEAE70120A0715D4684F803A034
:1005A000062000F02BFF0A2000F028FFDEE71922CA
:1005B0002946A54800F0CAFD98F8180000287CD00C
:1005C00098F80000062873D2DFE800F072030B46AB
:1005D000464940F2044000880290D8F80410814255
:1005E00066D098F809104FF00109404601295FD103
:1005F000D0F80A1019B995498969C0F80A1000267F
:10060000804617E0072000F0F9FED7F80E00B84644
:10061000871B402F00D94027A9193A468C48193129
:1006200000F094FDD8F80A003A4630448849FFF7B4
:10063000DDFD3E44D8F80E004746B042E2D8397896
:10064000012935D14FF0E0220906C2F88011D7F810
:100650000A00FFF7F9FD2BE04FF001092BE098F8B5
:1006600009104FF00109032925D17149794A002663
:100670000B68136017E07BE0072000F0BFFED7F89F
:100680000E00871B402F00D94027A9193A46704811
:10069000193100F05BFD66483A46006881196C48E4
:1006A00000F043FD3E44D8F80E004746B042E3D880
:1006B00098F8180008B1464600E01CE098F80800D9
:1006C000C00613D56349012202A8C1F800B005F1A4
:1006D0001801CDF808A000F019FD307820B1C8212C
:1006E0004FF47A7001F0F1F8307E20B1307A800753
:1006F00001D5FFF705FED8F80E001B35054452481A
:1007000000F058FD30B30220A07141485D4680F8EA
:1007100000A00B2000F072FEB9F1000F1AD03A4A87
:100720004FF00009916842F2107093685B1A83429F
:10073000FBD34FF42F714FF47A7001F0C6F83148B3
:10074000406D400502D50020099001E0099808B9E4
:10075000FFF7D6FDE078401CC0B2E0700C2802D351
:100760000120A07014E7A07800283FF413AF0FE732
:100770000120207002F0B6F9012002F074F924483B
:1007800000780028F1D0002105A800F031FC0028F5
:10079000EBD084F806A05D4684F803A0E6E61D4C85
:1007A0000026FF202660A680A671607101F06BF91B
:1007B00000F0C4FEFFF701FEFFF7E8FD00F0E4FDE6
:1007C000002000F01BFE01F0B5F902F05DFB01F026
:1007D0006FFA01F03DFAFFF717FE90B1042000F028
:1007E0000DFE084F7869084D800440D4FFF723FEC2
:1007F00038B1FFF720FE20B1FFF71DFE08B104203D
:100800002AE03CE0008009200000094080841E00AE
:1008100068000010BC00001046000000257325642D
:10082000000000000CED00E00000FA05AC00001034
:10083000B80000109C0000109400001098000010F8
:100840006101001060000010480100106C590000A8
:10085000D91B0010B000001000F0D0FDA8681C49A2
:100860007A69920403D4AA68121A8A42F8D3A86853
:1008700042F21071AA68121A8A42FBD3667100F024
:1008800037FC00F0A3FC80B1FFF7E5FC68B1022063
:1008900000F0B4FD94F90500401C03D10D488069B7
:1008A000FFF7D2FC0120607004E0022000F0A6FDFA
:1008B00066706671FFF7A8FD40B14021064804F05C
:1008C00076FC4022D101044800F02FFCFFF7F9FD2F
:1008D00080841E006C590000D91B00102DE9F047E0
:1008E000FE4A00234FF40077156A4FF4FF79C5F3F1
:1008F0000724DFF8ECA34FF4E05CDFF8E883FA4E5E
:1009000025E0B84216D213280CD014280CD0484544
:100910000CD0A0F58072FF3A0AD03E2813D81AF8FE
:10092000002011E0EAB20FE022460DE055220BE074
:10093000AA2209E0604506D208EB0002A2F5805227
:1009400092F8002E00E00022F254401C5B1C8B4207
:10095000D7D3BDE8F08770B5E04D2C6B402C00D9A3
:100960004024E86AE96902198A4202D90C1A042172
:1009700069702146FFF7B2FF2246DB49822002F070
:100980007CF9E86A2044E862286B011BD748296398
:100990008268A2EB0402826005D06978022901D046
:1009A0000021017370BD03216970F9E7CF4910B5CB
:1009B000CF4808600D22822002F05FF9C749052068
:1009C000487010BD70B50D46CA49496D490521D41E
:1009D000B0F5007F1ED3C849C04CB0F5E05F1AD215
:1009E0008A68A369D21AC54B9A4204D38968A16167
:1009F000002161606161BD4900235F39B94A07E0A8
:100A0000C4181444CE5CA4F580545B1C84F8006EBA
:100A1000AB42F5D370BD626922B98A68A2618A6867
:100A20006261A060B64A5279002AF3D18A6863698C
:100A3000D21AB44B9A421CD2B34B01221A708A6864
:100A4000A26189686161A168401A6168884203D91E
:100A5000616A884200D26060062000F0CFFC6168C5
:100A60002A46BDE87040A14801F500515F3800F00A
:100A70005CBBBDE870400C2000F0C0BC10B5974CCA
:100A8000A178E06A4218E1698A4206D9081AA07082
:100A900005206070022002F0ABF8A178E06AFFF751
:100AA00091FFA178E06A0844E062206B421A8F4807
:100AB00022638368A3EB0101816002D0617805297C
:100AC00004D100210173BDE810406FE710BD2DE98E
:100AD000F041824CA178E06A4218E1698A4206D965
:100AE000081AA07005206070022002F081F87F4D86
:100AF0000021A0787C4B5F3DE26A08E056186F5CED
:100B00009E5DBE4202D00021A16202E0491C8142EA
:100B1000F4D31118E162216B0A1A744922638B68BD
:100B2000A3EB0000886002D06078052808D1A06A95
:100B300020B100200873BDE8F04137E70120F9E754
:100B4000BDE8F081694810B51F38D0F81110027D5A
:100B500009BA21F0FF011143604A4902D162C18AFA
:100B600049BA49021163806888420CD0822002F0A1
:100B70003FF8022002F03CF85C4902200873FFF7BE
:100B800015FF002010BD012010BD70B55748574D0E
:100B90001F380224816829B1007B000607D4022097
:100BA00002F026F82C73FFF701FF002070BD012032
:100BB00070BD10B54D48494C1F388068A1788842F7
:100BC00000D2A0704949A2785F39822002F055F81E
:100BD000032060704548A2788168891A81600021ED
:100BE000017310BD414810B51F38816839B1007BD1
:100BF000000601D5822000E0022001F0F9FF3B4908
:100C000000200873BDE81040D0E610B5FFF7BDFF27
:100C100000281FD0354870215F3802220170002162
:100C200041708270C1700171417181710A22C2717B
:100C3000017241728172C1723022027301224273C9
:100C40008173C17301744174244912208870BDE816
:100C50001040AEE710BD1CB5FFF797FF00286AD023
:100C60002A480A2206210388684600F025FA1F4810
:100C700000225F3880230270437082700121C170AE
:100C80002021017143718271C2714122027254228A
:100C900042724F2282724C22C2720173417381737D
:100CA000C1734622027450234374722383746923F0
:100CB000C3746E230375742343758175C2756C22EA
:100CC000027661224276732282766822C2760177AA
:100CD00041778177C1779DF8011019E07800001005
:100CE0002C59000061010010D91B0010C01B00101E
:100CF000555342530080092000000940A08601009E
:100D0000BC00001020A107006800001004040000CF
:100D100080F820109DF8021080F821109DF8031033
:100D200080F822109DF8041080F82310DE4924205A
:100D30008870FFF73EFF1CBD10B5FFF726FF0028A7
:100D40000CD0DA4803210170002141708170C1701C
:100D5000D54904208870BDE810402AE710BD10B5C1
:100D6000FFF713FF002810D0D048002106220170A1
:100D700042708170C170017141718171C171CA4944
:100D800008208870BDE8104013E710BD10B5FFF7CC
:100D9000FCFE002815D0C44AC448116A491E0B0E37
:100DA00003700B0C43700B0A8370C170002101713A
:100DB000417102238371C17108209070BDE8104019
:100DC000F7E610BD10B5FFF7E0FE002819D0B748D0
:100DD0000021B54B0170417081700822C2701A6AFF
:100DE000140E0471140C4471140A8471C27102222D
:100DF000027241728272C1720C209870BDE810407C
:100E0000D7E610BD2DE9F041A74DA84C0021A878E8
:100E10004034A64A02E0535C6354491C03468142B5
:100E2000F9D31F2B72D12068A14988426ED19F4E01
:100E300060685F364FF001087060A068B060607B4A
:100E400018B9A07B08B1102802D986F80C8059E0A7
:100E5000E07B1E28F9D00FDC12282ED005DC48B329
:100E60000328F2D1BDE8F041CFE61528EDD01A28CD
:100E7000EBD1BDE8F0415FE702272A2828D010DC3B
:100E800023281DD025281ED02828DED1FFF75AFEA2
:100E9000002826D0207B000618D56F70BDE8F041F1
:100EA00059E52F281ED05528CFD05A28CDD1BDE8DE
:100EB000F04154E7BDE8F04194E6BDE8F041CAE6F0
:100EC000BDE8F0417EE7BDE8F0415FE7022016E0B3
:100ED000FFF738FE002804D0207B00060ED485F8EA
:100EE00001802DE6FFF72EFE0028FAD0207B0006B9
:100EF00004D485F80180C5F8288021E6822001F01D
:100F000077FE3773BDE8F04150E5FFE7822001F03E
:100F10006FFE022001F06CFE0620687010E6624849
:100F200010B54178022908D003290ED004290FD02A
:100F3000052901D10021417010BD5C484030C07BC3
:100F40002828F9D1BDE8104005E5BDE810402DE5A1
:100F5000822001F04DFEF8E710B55449022001F05F
:100F60005BFE51498870487858B101280CD00220A6
:100F700001F03EFE4D4902205F310873BDE810408C
:100F800014E5BDE810403DE748484030C07B2A28C2
:100F900004D02F2805D1BDE8104098E5BDE81040E9
:100FA0006CE510BDFFB50246002002EB420501468C
:100FB0004FF440566C4603AA6B1844F82130B342F4
:100FC00002DD002004B0F0BD3A4F07EB6307DB07FA
:100FD0003F78575401D03B095354535C8F0003F0C2
:100FE0000F035354BB40491C18440329E4DBE9E7D1
:100FF000F0B506460020034602462E4C4FF400771B
:1010000000E05B1CF55C45B102EB030CA4440CF55D
:10101000805C9CF800C8AC45F3D0032B3FD302F5AD
:10102000C0502044037F457FC67F03EB0523857FA7
:101030002D0405EB06652B4451EA03052BD021B99D
:101040001949496840318B4225D8184B00216C332F
:101050005518254405F5805595F800585D54491CF0
:101060000C29F5D3817EC27E01EB0221027D407DF9
:10107000120402EB00600C182046FFF793FF40F6C5
:10108000F57501E0FFF78EFFC11EA942FAD3A0F566
:101090007061FF3901D00020F0BD2046F0BD203244
:1010A000BA42AFD3F0BD000078000010611B001001
:1010B0005553424361010010FFB5ACA60446E1CE92
:1010C0008DE8E100022902DA002004B0F0BD6018CA
:1010D000002100F8011D6946B3FBF2F502FB15354E
:1010E000B3FBF2F34D5D00F8015DA042F4D8ECE7EC
:1010F00010B503F095FF03F07FFFA0494FF40052B5
:10110000C1E90020A0F5F420886010BD70B5034649
:1011100008468D189949002449688D4200D9881ADB
:10112000194603F0CCFF204670BDF8B51446934E27
:101130000A460B19716800258B4200D90A1B034629
:101140000094306803F0E6FF2846F8BD10B50B4662
:1011500001460024184603F086FF204610BD2DE905
:10116000FC410746002090460E46ADF800000446BC
:101170000EE0351B402D00D9402539192A468048FC
:10118000FFF7E4FFAAB27E496846FEF7B9FF2C4498
:10119000B442EED33919424601A8FFF7D7FFBDF894
:1011A0000000BDF80410884202D10120BDE8FC8196
:1011B0000020FBE70021425C12B9491C1829FAD330
:1011C000182901D000207047012070472DE9F04117
:1011D0006A4C00270C3488B0A770E770DFF8A48150
:1011E0004FF40056277101251922314601A8FFF757
:1011F000ADFF022216213046FFF7B1FF00287DD057
:10120000DDF81210022206F11900FFF7A8FF0028EE
:1012100074D09DF80400062829D2DFE800F02903E5
:101220000329291CD8F87410DDF80E30491C8B42B4
:101230001DD2D8F87420DDF80E30D21ADDF8123045
:10124000521C9A4213D3DDF80E20DDF812301A44F6
:101250008A420CD80CE0DDF81210B1F5F42F00D959
:10126000A570DDF81610C1F30B41702900D0A570F0
:10127000012803D0022801D0052839D1022206F224
:101280001D4168460097FFF761FF0099029889B2F7
:10129000884200D0A570012206F2254168460097D9
:1012A000FFF754FF0099BDF80500C9B2884200D08D
:1012B000A5709DF8040002281AD1042206F24941C3
:1012C00068460097FFF742FFDDF816000099884254
:1012D00000D0A570012206F24D4168460097FFF745
:1012E00035FF00989DF80710C0B2814200D0A5706C
:1012F0009DF81C00401EFE2802D200E01EE0A570F2
:10130000BDF80500A0F57F41FF3901D0452802D185
:101310009DF8070020B901A8FFF74CFF00B9A570A0
:10132000DDF812001B36064401A8FFF743FF30B179
:10133000E07880B1217988420DD012E0A5709DF847
:101340001C0010B92079401C2071E078401CC0B20C
:10135000E0700C2801D3A57003E0A07800283FF4CA
:1013600043AFA07808B0BDE8F081000030313233DF
:10137000343536373839414243444546B0000010D1
:10138000D91B0010E4590000002070476949C207CA
:1013900002D04FF000728A67800702D54FF080605C
:1013A0008867002070476349C20702D04FF000727F
:1013B000CA67800702D54FF08060C8670020704779
:1013C000014600205B4ACB0703D0536F9B0100D539
:1013D0000120890704D5516F490101D540F0020071
:1013E000704710B50446FFF7EBFF0346FFF7DBFF3E
:1013F00024EA0300FFF7CAFF002010BD70B54E4B72
:1014000050B15968042403250226052907D2DFE8D4
:1014100001F0072B4A718E0000205860986070BD63
:10142000042807D0052809D0012402287AD00128F1
:1014300008D00FE00320FFF7B6FF46E0BDE870409C
:101440000120B0E70320FFF7AEFF0BE0FFF79EFFA0
:101450005C6070BD0E28FCD10320FFF7A4FF0220C2
:10146000FFF794FF0120F1E706280AD0032810D0E7
:101470000A2813D0092811D00D280FD00C28D9D054
:1014800070BD0320FFF78FFF0220FFF77FFF5E6034
:1014900070BD0320FFF787FF012027E00320FFF73F
:1014A00082FF022012E0062813D00A281AD0092849
:1014B000C8D00C28BED00D28F0D00F28E8D10320CA
:1014C000FFF771FF0220FFF761FF0120BDE87040C8
:1014D0005CE7986810F01F0F00F101009860D7D109
:1014E00002201BE00320FFF75EFF0220FFF74EFF04
:1014F0005D6070BD072806D00A289BD00B2811D04C
:1015000009289FD070BD0220FFF74DFF986810F0AA
:101510003F0F00F101009860F4D10120BDE8704058
:101520005FE7FFE70320FFF73EFF02208EE7062874
:10153000A7D08FE700800920D0000010F0B5AB499C
:10154000012041F8680F0326C1F80862C1F80C6257
:101550000920C1F89800C1F89C00C1F8A000C1F8AA
:10156000A400C1F8A8001022CA66A14853048363EE
:10157000036A43F4001303620D238B668B67002319
:10158000C1F8AC3020248465046C44F02004046469
:1015900041F8243C54038461046844F4003404603A
:1015A000C1F8803094058463046A44F08064046266
:1015B000C1F88430D4058463046A44F00064046292
:1015C000C1F8B4208024C465056C25F0800505644D
:1015D0009025C1F894504FF0004EC0F83CE0076AE7
:1015E00027F0004707624A67D704C763076A27F4F2
:1015F00000070762C1F82822C0F8BC20D0F8A0700C
:1016000027F01007C0F8A070012741F8087C41F8C6
:101610000C7C41F8047C0E670526CE6741F8607C9F
:10162000112641F85C6C0226C1F8B8601227C1F897
:10163000BC7040F2822741F8447C4FF09A0C41F88C
:1016400048CC41F84C7C41F8542D2027876107682D
:1016500047F0200707604A6040278761D0F800C044
:101660004CF0400CC0F800C0CA614FF4805CC0F878
:101670001CC0D0F800C04CF4805CC0F800C04FF033
:10168000010C41F85CCF41F804CCC1F880204FF048
:10169000805CC0F838C0D0F820C04CF0805CC0F846
:1016A00020C0C1F884204FF0005CC0F83CC0D0F8E6
:1016B00020C02CF0005CC0F820C041F83C5C550212
:1016C000C561056825F400550560CB65D503C56384
:1016D000056A25F40025056241F8384C9402C4617E
:1016E000046844F480440460C1F81432C0F8BC605B
:1016F000D0F8A04044F00204C0F8A040C1F8743112
:101700005405C467046E44F000740466C1F878316F
:1017100094058467046E44F0806404668A24C1F8EA
:10172000884008248C659503C563046A44F48024CA
:101730000462C1F8B8209401C465046C24F4806488
:101740000464322441F81C4C302641F8286CC561F1
:10175000056825F48025056041F8244C41F8204CAB
:1017600041F8184CC1F8BC40C1F8C040C1F8C440B1
:10177000012441F8104F4C600C610C624C628C6289
:1017800041F8384F4C608C60CC600B66C765036CC9
:1017900043F04003036441F8A82CC261036843F09E
:1017A00010030360C1F8C0219306C0F89C3050F8C4
:1017B000803F43F080430360C1F8C421C0F818E0C3
:1017C000026842F0004202600A480B4AB8390068D9
:1017D000904201D1012003E0084A904204D18120C7
:1017E00041F8B80F8860C860F0BD000000C002403A
:1017F00000800920CC000010473F1927473F1947B8
:101800004D4900200867C86002224A618861302281
:10181000CA634A498A684A49C1E9002049490860BF
:1018200049490860784649490860002070472DE919
:10183000F04341F288320024424F434E434B9042E2
:1018400008D8642800D228B942F21072914201D817
:10185000052907D2862038607846346018608620D3
:10186000BDE8F083DFF8D490D9F80850344AD2F8B4
:1018700000C0A5EB0C05D2F804C00CEB4C08C8EB7B
:10188000CC1CB5EBCC0F06D205203860784634600E
:1018900018600520E4E7284D4FF0020CC5F804C09D
:1018A00048B1DFF8AC80B8FBF0F04010A861C5F893
:1018B00004C001206860D9F80800C2E900013C605A
:1018C0007846346018600020CAE770B51C4C0025CB
:1018D0000E466560FFF7ABFF1A49000601D50868A0
:1018E00070BD164B06EB46022068C2EBC6129E681E
:1018F000361AB6EBC20FFAD30F4802224260C26B0F
:1019000002F0FE02C2636560E9E70C4880680C499A
:101910000A68801A4A6802EB4203C3EBC212B0EBBA
:10192000C20F08D3044802224260C26B02F0FE02DA
:10193000C2630020486070470080004000000940FA
:10194000E00000106C000010700000107400001027
:1019500080C3C901F0B57248D0F804114FF00002FD
:10196000CB05704928D4D0F80C31DC076E4B03D07E
:10197000D0F8A041640660D5D0F80441E40605D053
:10198000D0F8044104F01F04B3FBF4F40C60D0F869
:10199000A851ED060ED0D0F8A85105F01F05B3FBF5
:1019A000F5F34B60D0F8003103F001035B1CB4FB8E
:1019B000F3F331E00023F4E7D0F88830DB053CD5C1
:1019C000D0F80C31DB0703D0D0F8A0315B0634D55A
:1019D000D0F88830D0F8044103F01F0314F01F053D
:1019E000D0F8A841D0F8006104F01F0406F0010609
:1019F00003F1010306F1010603D04B4F5F43B7FB30
:101A0000F5F50D6024B1484F7B43B3FBF4F300E0E0
:101A100000234B60B5FBF6F3C1F80830D0F808316D
:101A2000DB05D0F808311CD513F01F0303D0042BBD
:101A300007D0062B05D0CA60F0BD0A604A608A60F4
:101A4000ECE7D0F88820D0F8083102F01F02D0F877
:101A50000C0103F01F033448521C4243B2FBF3F065
:101A60000FE09B05E7D5D0F80C21D20702D0D0F8C3
:101A7000A80001E0D0F888002B4A00F01F00401CAD
:101A80005043C860F0BD264810B42021C0F8A01112
:101A9000D0F8A0114906FBD50121C0F80C1109228C
:101AA000C0F88420C0F88010AA22C0F88C205523EA
:101AB000C0F88C30D0F888406405FBD52324C0F8EA
:101AC000A440C0F8A010C0F8AC20C0F8AC3000BFF3
:101AD000D0F8A8205205FBD540F20112C0F804212D
:101AE00040F20122C0F80821C0F800110221C0F81C
:101AF000B4110421C0F8A8110C49C0F8C410002189
:101B0000C0F8C811D0F8B02142F00302C0F8B021EB
:101B100045F23A0202600648016010BC1AE7000074
:101B200000C00F40E8000010001BB700FE9FF8F750
:101B300008ED00E01849174808601849886842F223
:101B400010728B681B1A9342FBD300207047124916
:101B50000A6822F080720A600A68012322F0FF02FC
:101B600083401A4342F08070086048680028FCDA1D
:101B70000A6822F080720A6080B2704710B5EFF3F5
:101B8000108101F0010472B6FFF7E1FF002C00D1D3
:101B900062B610BD00012000004003400000094073
:101BA000FEE7FEE7FEE7FEE74FF40050704730B473
:101BB00020F07043094C000F54F820401846A4460A
:101BC00030BC604730B420F07043044C000F403408
:101BD00054F820401846A44630BC60475C5A0000C8
:101BE00008B5012269462D48FFF7E1FF9DF8000086
:101BF00008BD01B5012269462848FFF7E3FF08BD8B
:101C00004420FFF7F6FF26498868264A8B681B1A8E
:101C10009342FBD324494FF480408861FEE710B51E
:101C20002248214A00210378526B4FEA02321BB14D
:101C3000002A00DA017010BD002A02DB8168491C0D
:101C400004E08268642A01D9FFF7DAFF816010BDE1
:101C50002DE9F041154C00252570FFF7C1FF104B11
:101C6000012299684CF250369F687F1AB742FBD325
:101C70000D494B6B1B0302D5552803D00AE05528AC
:101C800000D03AB15520FFF7B4FF01206560207005
:101C9000BDE8F0814FF480408861FEE72800002015
:101CA00000000940400D030000800920F8000010EA
:101CB00070B500BF00BF00BF00BF00BF00BF00BFC6
:101CC00000BF00BF00BF00BF00BF00BF00BF00BF1C
:101CD00000BF00BF00BF00BF00BF00BF00BF00BF0C
:101CE00000BF00BF00BF00BF00BF00BF00BF00BFFC
:101CF00000BF2025FB4CE561062001F0D8F8A56166
:101D000000BF00BF00BF00BF00BF00BF00BF00BFDB
:101D100000BF00BF00BF00BF00BF00BF00BF00BFCB
:101D200000BF00BF00BF00BF00BF00BF00BF00BFBB
:101D300000BF00BF00BF00BF00BF00BF00BF00BFAB
:101D400000BF00BF00BF00BF00BF00BF00BF00BF9B
:101D500000BF00BF00BF00BF00BF00BF00BF00BF8B
:101D600000BF00BF00BF00BF00BF00BF00BF00BF7B
:101D700000BF00BF00BF00BF00BF00BF00BF00BF6B
:101D8000E561052001F093F8002001F090F8A561CD
:101D900000BF00BF00BF00BF00BF00BF00BF00BF4B
:101DA00000BF00BF00BF00BF00BF00BF00BF00BF3B
:101DB00000BF00BF00BF00BF00BF00BF00BF00BF2B
:101DC00000BF00BF00BF00BF00BF00BF00BF00BF1B
:101DD0008107C54827D50121017000BF00BF00BFA2
:101DE00000BF00BF00BF00BF00BF00BF00BF00BFFB
:101DF00000BF00BF00BF00BF00BF00BF00BF00BFEB
:101E000000BF00BF00BF00BF00BF00BF00BF00BFDA
:101E100000BF00BF00BF00BF00BFE561012001F0AF
:101E200046F8802026E00221017000BF00BF00BFFD
:101E300000BF00BF00BF00BF00BF00BF00BF00BFAA
:101E400000BF00BF00BF00BF00BF00BF00BF00BF9A
:101E500000BF00BF00BF00BF00BF00BF00BF00BF8A
:101E600000BF00BF00BF00BF00BFE561012001F05F
:101E70001EF8402001F01BF8A56100BF00BF00BFA5
:101E800000BF00BF00BF00BF00BF00BF00BF00BF5A
:101E900000BF00BF00BF00BF00BF00BF00BF00BF4A
:101EA00000BF00BF00BF00BF00BF00BF00BF00BF3A
:101EB00000BF00BF00BF00BF00BF00208B4908600B
:101EC0008B49086078468B490860002070BD2DE979
:101ED000F74F864D864E874F5FEA020B044612D0BD
:101EE000814820217F4A00784FF0820A012812D0D1
:101EF00002287DD02420C5F800A0306078463860E4
:101F00008220BDE8FE8F8620286009203060784658
:101F100038608620F5E700BF00BF00BF00BF00BFEC
:101F200000BF00BF00BF00BF00BF00BF00BF00BFB9
:101F300000BF00BF00BF00BF00BF00BF00BF00BFA9
:101F400000BF00BF00BF00BF00BF00BF00BF00BF99
:101F500000BF00BF00BF88469146D161052000F058
:101F6000A6FF002000F0A3FF4A46C9F8188000BF72
:101F700000BF00BF00BF00BF00BF00BF00BF00BF69
:101F800000BF00BF00BF00BF00BF00BF00BF00BF59
:101F900000BF00BF00BF00BF00BF00BF00BF00BF49
:101FA00000BF00BF00BF00BF00BF00BF00BF00F008
:101FB000F100802803D00320C5F800A09DE700BFF2
:101FC00000BF00BF00BF00BF00BF00BF00BF00BF19
:101FD00000BF00BF00BF00BF00BF00BF00BF00BF09
:101FE00000BF00BF00BF00BF00BF00BF00BF00E0D8
:101FF00019E000BF00BF00BF00BF00BF00BF00BFAF
:1020000000BFC2F81C80032000F051FF200A00F03E
:102010004EFF204600F04BFF5946019800F059FF53
:102020004046494635E000BF00BF00BF00BF00BFCB
:1020300000BF00BF00BF00BF00BF00BF00BF00BFA8
:1020400000BF00BF00BF00BF00BF00BF00BF00BF98
:1020500000BF00BF00BF00BF00BF00BF00BF00BF88
:1020600000BF00BF00BF89469046D161032000F049
:102070001EFF002000F01BFFC4F3072000F017FF35
:10208000E0B200F014FF5946019800F022FF4846E4
:102090004146886100BF00BF00BF00BF00BF00BF56
:1020A00000BF00BF00BF00BF00BF00BF00BF00BF38
:1020B00000BF00BF00BF00BF00BF00BF00BF00BF28
:1020C00000BF00BF00BF00BF00BF00BF00BF00BF18
:1020D00000BF00BF002028603060784638600020D4
:1020E0000FE7000000800920040100106C000010C0
:1020F00070000010740000102DE9F74FDFF88C938A
:10210000DFF88CA3DFF88CB384B01500884616D0B6
:102110000320E14E0290E14800270078012819D001
:1021200002287DD082202421C9F80000CAF80010BE
:1021300079468220CBF8001007B0BDE8F08F8621E9
:10214000C9F800100921CAF8001079468620CBF89A
:102150000010F1E700BF00BF00BF00BF00BF00BF1D
:1021600000BF00BF00BF00BF00BF00BF00BF00BF77
:1021700000BF00BF00BF00BF00BF00BF00BF00BF67
:1021800000BF00BF00BF00BF00BF00BF00BF00BF57
:1021900000BF00BF2024F461062000F088FEB46177
:1021A00000BF00BF00BF00BF00BF00BF00BF00BF37
:1021B00000BF00BF00BF00BF00BF00BF00BF00BF27
:1021C00000BF00BF00BF00BF00BF00BF00BF00BF17
:1021D00000BF00BF00BF00BF00BF00BF00BF00BF07
:1021E00000BF00BF00BF00BF00BF00BF00BF00BFF7
:1021F00000BF00BF00BF00BF00BF00BF00BF00BFE7
:1022000000BF00BF00BF00BF00BF00BF00BF00BFD6
:1022100000BF00BF00BF00BF00BF00BF00BF00E0A5
:102220006AE000BFF461022000F041FE0498000A59
:10223000009000F03CFE049800F039FE294640462C
:1022400000F03CFEB46100BF00BF00BF00BF00BF94
:1022500000BF00BF00BF00BF00BF00BF00BF00BF86
:1022600000BF00BF00BF00BF00BF00BF00BF00BF76
:1022700000BF00BF00BF00BF00BF00BF00BF00BF66
:1022800000BF00BF00BF00BF00BF00BF00BF00BF56
:1022900000BF00BF00BF00BF00BF00BF00BF00BF46
:1022A00000BF00BF00BF00BF00BF00BF00BF00BF36
:1022B00000BF00BF00BF00BF00BF00BF00BF00BF26
:1022C00000BF00BF00BFF461032000F0F0FD0098E4
:1022D00000F0EDFD049800F0EAFD002409E0002084
:1022E00000F0E5FD18F80410C0B2814200D00127CB
:1022F000641CAC42F3D392E000BF00BF00BF00BF3C
:1023000000BF00BF00BF00BF00BF00BF00BF00BFD5
:1023100000BF00BF00BF00BF00BF00BF00BF00BFC5
:1023200000BF00BF00BF00BF00BF00BF00BF00BFB5
:1023300000BF00BF00BF00BF2024F461022000F0F6
:10234000B6FD002000F0B3FD0498C0F30720039011
:1023500000F0ADFD0498C0B200F0A9FD294640464A
:1023600000F0ACFDB46100BF00BF00BF00BF00BF04
:1023700000BF00BF00BF00BF00BF00BF00BF00BF65
:1023800000BF00BF00BF00BF00BF00BF00BF00BF55
:1023900000BF00BF00BF00BF00BF00BF00BF00BF45
:1023A00000BF00BF00BF00BF00BF00BF00BF00BF35
:1023B00000BF00BF00BF00BF00BF00BF00BF00BF25
:1023C00000BF00BF00BF00BF00BF00BF00BF00BF15
:1023D00000BF00BF00BF00BF00BF00BF00BF00BF05
:1023E00000BF00BF00BFF461032000F060FD0020CB
:1023F00000F05DFD039800F05AFD0498C0B200F0B3
:1024000056FD002409E0002000F051FD18F80410EA
:10241000C0B2814200D00127641CAC42F3D320201B
:10242000B06100BF00BF00BF00BF00BF00BF00BF62
:1024300000BF00BF00BF00BF00BF00BF00BF00BFA4
:1024400000BF00BF00BF00BF00BF00BF00BF00BF94
:1024500000BF00BF00BF00BF00BF00BF00BF00BF84
:1024600000BF4FB10298401E02907FF454AE82200C
:102470000421C9F8000059E60020C9F80000794697
:10248000CAF80000CBF8001056E600006C000010FF
:10249000700000107400001000800920040100107A
:1024A000FA4800214FF00112818001704170C0E9AB
:1024B00002217047F5491C31002000F0ADBB10B57A
:1024C000F24C1434A288402A00D94022802021688E
:1024D00000F0D3FB216801442160A188081AA08084
:1024E00010BD10B5E94C00201434216800F094FBB5
:1024F000216801442160A188081AA08010BD002233
:102500001146802000F0B9BBE149002000F084BBF7
:1025100070B5DE48DD4D1C3005F11405007810F073
:102520001F040AD0D949DA4B01F11C004A7800791E
:10253000012C06D0022C26D109E0D448001D2860C9
:102540001DE002B3897888421DD2002015E000F01A
:102550008F04200605D504F00F064FF48030B040FC
:1025600001E00120A0400AB922070CD18A6802428A
:1025700009D0C9680142E8D0012018802B60FFF71C
:102580009EFF012070BD002070BD024670B5BF489F
:10259000BE4C1C30017811F01F030146498804D05D
:1025A000012B29D0022B27D111E0012924D132B1EE
:1025B000012000F0CCFAA08840F0020005E00020E5
:1025C00000F0C5FAA08820F00200A08021E0007988
:1025D00000F08F00030605D500F00F034FF480359F
:1025E0009D4001E00125854063782BB1030703D0AE
:1025F000A3682B4200D009B1002070BD22B100F0C9
:10260000F7FAE068284303E000F0FCFAE068A8432A
:10261000E060012070BD9D4810B51C30007810F0BE
:102620001F0F9A4800F11C00C0782AD19749143135
:10263000012807D001F108020228937806D0032868
:102640001FD112E093480860122012E09248002245
:1026500004E004780CB144882044521C9342F8D121
:10266000027872B10860408803E08C481844086022
:1026700000788A88824200D98880FFF720FF0120F5
:1026800010BD002010BD2DE9F84F804F00201C37F1
:102690000090B8787D4E4FF000094FF0010A4FF4DA
:1026A000803B00286BD07C4C65E06078022804D029
:1026B000042841D005285CD141E06179B878814295
:1026C00038D170702079B0707049002011F110017C
:1026D00001F80090401C0428FAD301254FEA0608AF
:1026E0000AFA05F0D8F80810084202D0284600F08F
:1026F0006BFAD8F808100BFA05F0084203D045F041
:10270000800000F061FA6D1C102DE9D34FF001102C
:10271000C8E90209012000F01BFAE0794006B8F888
:10272000040002D540F0010001E020F00100A8F80B
:1027300004001EE060881DE0E078009019E0009839
:10274000B8B9A07800F08F05280604D505F00F0170
:102750000BFA01F001E00AFA05F0B16801432046E6
:10276000B16000F00AFA284600F024FA284600F08A
:1027700035FA207804442078002896D11FE086F8A6
:10278000019001245546D846B16805FA04F0084284
:1027900002D0204600F018FAB16808FA04F00842A6
:1027A00003D044F0800000F00FFA641C102CEBD32F
:1027B0004FF00110C6E90209002000F0C9F9B8780D
:1027C0007178884202D10120BDE8F88F0020FBE734
:1027D0002DE9FC5F2D4D00273E466878BB46B84684
:1027E000002871D0BA462C4C05F11C0968E06078CD
:1027F000022804D0042808D005285FD119E06079A8
:10280000697888425AD0608859E0A77899F804100E
:10281000E6784FF00008B94250D199F80200B04272
:102820004CD11A484FF0010A103010F807B0C655C5
:1028300044E099F80410B94240D1A17801F08F0129
:102840000191090605D5019901F00F024FF480317D
:1028500001E0019A01219140009199F80200B042F3
:102860001ED1A8680843A860E96800988143204603
:10287000E96000F082F9019800F09CF9019800F0FD
:10288000ADF9009948EA010818E0000008010010BD
:10289000441D00105C5B00006E5B00008F5B00005D
:1028A0005E450BD118EA010F08D1A8688843A860DB
:1028B000E8688843E860019800F086F920780444CD
:1028C0002078002893D15046BDE8FC9F2DE9F041C7
:1028D000494C0027A4F108062178A4F11C0508281A
:1028E00063D2DFE800F06204647262628381FFF702
:1028F000E1FD2078C00900F05CF9E088B080207824
:10290000C0F34111F1BB61780C294AD2DFE801F034
:102910000609490B49101A1D1F253142FFF7F8FD22
:102920004DE0002000E00120FFF72FFE50B306E04D
:1029300010F01F0F35D1A07840F080002870BDE85E
:10294000F041DCE5FFF767FE39E000202AE010F0F7
:102950001F0F26D128481B381AE010F01F0F20D176
:10296000FFF791FE70B1FFF7CAFDBDE8F04100F03E
:1029700077BA00F01F00012813D1687810B12079D0
:10298000A97800E00DE088420BD21B490C390844BD
:1029900030601CE000F01F00012802D1FFF718FF93
:1029A000C4E7802000F024F9B780BDE8F081080674
:1029B00008D4B0880028F8D0FFF793FDB08800282D
:1029C000EFD0F2E7BDE8F0419EE5080602D5BDE88C
:1029D000F04174E528780106E7D500F07F00287003
:1029E000BDE8F04100F054B8802000E00020BDE8D0
:1029F000F04100F007B90000240100100146000773
:102A0000C00E090600D5401C7047E1491022C1F8EC
:102A10000822C1F8100200BFD1F80002C006FBD5A1
:102A20007047DB4A1023C2F80832C2F8100200BF18
:102A3000D2F80002C006FBD5C2F80832C2F8101264
:102A4000D2F80002C006FBD57047D1493022C1F848
:102A50000822C1F8100200BFD1F800028006FBD5A1
:102A6000D1F81402704710B5040001D0012000E035
:102A700000204FF4807141EA0041C648FFF7D1FFC2
:102A8000C5494FF480200CB1886310BDC86310BDE8
:102A900030B5C249C24D41EA004421462846FFF7FD
:102AA000C0FF21462846BDE83040BAE7B8480021BB
:102AB000C0F848124021C0F84C120122C0F8482248
:102AC000C0F84C12D0F80012C905FBD54FF0FF3109
:102AD000C0F83812C0F83412C0F808120C21C0F83F
:102AE000041270472DE9F041FDF725FCAD4D1A2188
:102AF00029602A1D136831EA0303FBD1A44E002785
:102B00000123A94C142804DAE3670320C6F8100156
:102B100003E06367A367C6F810718A20C4F8F80061
:102B20002960106831EA0000FBD14FF0E0214FF03E
:102B30008070C1F880029D4B202283F80024C1F8E8
:102B40000001FFF7B3FFBDE8F0410020A0E77047A8
:102B500010B500B101204FF4807444EA004194485C
:102B6000FFF75FFF8A480321C0F84412D0F8001233
:102B7000C905FBD5C0F8084210BD10B502468078E3
:102B8000FFF73CFF8249D1F84432012484402343BB
:102B9000C1F84432C1F848029088C1F84C0200BF25
:102BA000D1F80002C005FBD54FF48070C1F80802CF
:102BB00010BD704700B5FFF721FF7E495DF804EBBB
:102BC00041EA004089132CE700B5FFF717FF794968
:102BD0005DF804EB41EA0040774922E700B5FFF7D2
:102BE0000DFF74495DF804EB41EA0040891318E7D2
:102BF00000B5FFF703FF6F495DF804EB41EA0040C1
:102C00006E490EE700B5FFF7F9FE6A495DF804EB7F
:102C100041EA0040891304E700F00F02012370B578
:102C200003EB82035A4AC2F8283200BFD2F820329E
:102C30001C05FBD5C3F309030024DD1C05E000BF20
:102C4000D2F8186241F8046B641CB4EB950FF7D30B
:102C50000021C2F8281241F24821C140C9070AD117
:102C6000FFF7CCFE4FF4A06141EA0040FFF7CDFE34
:102C70005348FFF7CAFE184670BD70B513460546A7
:102C8000434C00F00F00022202EB8000C4F828023F
:102C9000C4F824320020DA1C05E000BF51F8046BB0
:102CA000C4F81C62401CB0EB920FF7D30020C4F8AC
:102CB00028022846FFF7A2FE4FF4A06141EA004037
:102CC000FFF7A3FE3F48FFF7A0FE184670BD2DE9B1
:102CD000F0412F4DD5F80032C5F80832180721D53C
:102CE0002C48FFF792FE3848FFF7AFFEC10605D526
:102CF000FFF7DCFEBDE8F04100F0A3B8810705D581
:102D0000BDE8F04100F0010000F095B8010709D5D9
:102D1000400703D5BDE8F04100F09AB8BDE8F041A6
:102D200000F09DB8294E58074FF001071CD4BDE8AC
:102D3000F0810024D5F8302207FA04F10A4210D0BD
:102D40006008C5F8381200BFD5F800128906FBD517
:102D5000D5F81412E2070CD056F8201009B1032060
:102D60008847641C202CE5D3D5F830020028E0D138
:102D7000DDE73CB9490705D5316819B1012088471D
:102D80000124D7E756F820100029EAD00220E7E70F
:102D900000C008200005FE0000800920000180001E
:102DA0000005D000F4CF082000C0024018E000E089
:102DB0000005D800000540000001200000010100CE
:102DC0000005F2000005FA000002FE00005C0000B1
:102DD00070B5284C607820B30026274D012810D00C
:102DE00002280DD1A8686168401A2449884215D389
:102DF0002348406B400011D50120FFF734FE667078
:102E000070BDA8686168401A1E498842F8D3002046
:102E1000FFF729FEA86860600220607026700C2011
:102E200005E020780028EBD1012020700D20BDE8BE
:102E30007040FEF7E3BA002802D10E490120487025
:102E4000704710B5FFF72CFB0A490020487010BDF1
:102E500008480121417008498968416070477047FE
:102E60007047022803D0032803D1FEF758B8FEF7B5
:102E700073B870472C01001000000940A0860100C3
:102E80000080092040420F001848022101610722FA
:102E900002600022426142624160C168C906FCD4FE
:102EA00000E08168C1684907FBD4002070470F49E2
:102EB0008860C868C006FCD48868704700B50B46B7
:102EC000024603E012F8010BFFF7F1FF5B1EF9D297
:102ED00000BD00B50B46024604E00020FFF7E7FF07
:102EE00002F8010B5B1EF8D200BD00000000034099
:102EF0002DE9F047F84E80464FF080773068402447
:102F0000F64DB84249D100BF00BF00BF00BF00BFAF
:102F100000BF00BF00BF00BF00BF00BF00BF00BFB9
:102F200000BF00BF00BF00BF00BF00BF00BF00BFA9
:102F300000BF00BF00BF00BF00BF00BF00BF00BF99
:102F400000BF00BF00BFEC611520FFF7B0FF0020FD
:102F5000FFF7ADFF00F0FF09AC6100BF00BF00BF8D
:102F600000BF00BF00BF00BF00BF00BF00BF00BF69
:102F700000BF00BF00BF00BF00BF00BF00BF00BF59
:102F800000BF00BF00BF00BF00BF00BF00BF00BF49
:102F900000BF00BF00BF00BF00BF00BF00BF00BF39
:102FA00000BF00BF00BF00BF00BF00BF00BF00BF29
:102FB00000BF00BF00BF00BF00BF00BF00BF00BF19
:102FC00000BF00BF00BF00BF00BF00BF00BF00BF09
:102FD00000BF00BF00BF00BF00BFEC610620FFF7CD
:102FE00066FFAC6100BF00BF00BF00BF00BF00BFF5
:102FF00000BF00BF00BF00BF00BF00BF00BF00BFD9
:1030000000BF00BF00BF00BF00BF00BF00BF00BFC8
:1030100000BF00BF00BF00BF00BF00BF00BF00BFB8
:1030200000BF00BF00BF00BF00BF00BF00BF00BFA8
:1030300000BF00BF00BF00BF00BF00BF00BF00BF98
:1030400000BF00BF00BF00BF00BF00BF00BF00BF88
:1030500000BF00BF00BF00BF00BF00BF00BF00BF78
:1030600000BF00BFEC610120FFF721FF4FEA88009D
:10307000FFF71DFF3068B84202D14846FFF717FF3F
:10308000AC6100BF00BF00BF00BF00BF00BF00BFFA
:1030900000BF00BF00BF00BF00BF00BF00BF00BF38
:1030A00000BF00BF00BF00BF00BF00BF00BF00BF28
:1030B00000BF00BF00BF00BF00BF00BF00BF00BF18
:1030C00000BFBDE8F0872DE9FC5F8846044601A9F2
:1030D000834800F05AFB834D834E844FF0BB03209E
:1030E0008DF8000020098DF8010020018DF8020004
:1030F0004FF000098DF8039000BF00BF00BF00BF74
:1031000000BF00BF00BF00BF00BF00BF00BF00BFC7
:1031100000BF00BF00BF00BF00BF00BF00BF00BFB7
:1031200000BF00BF00BF00BF00BF00BF00BF00BFA7
:1031300000BF00BF00BF00BFDFF8A0B14FF0400AE2
:10314000CBF81CA004216846FFF7B8FE002400203D
:10315000FFF7ADFEC0B28DF8040000E003E018F800
:103160000410884208D082202860222030607846EF
:1031700038608220BDE8FC9F641CB4F5805FE6D314
:10318000CBF818A000BF00BF00BF00BF00BF00BF4A
:1031900000BF00BF00BF00BF00BF00BF00BF00BF37
:1031A00000BF00BF00BF00BF00BF00BF00BF00BF27
:1031B00000BF00BF00BF00BF00BF00BF00BF00BF17
:1031C00000BF00BFC5F800907846C6F80090386090
:1031D0000020CFE72DE9F0474FF0000900BF00BF06
:1031E00000BF00BF00BF00BF00BF00BF00BF00BFE7
:1031F00000BF00BF00BF00BF00BF00BF00BF00BFD7
:1032000000BF00BF00BF00BF00BF00BF00BF00BFC6
:1032100000BF00BF00BF00BF00BF00BF40252F4E52
:10322000F5619F20FFF743FE0020FFF740FE00F00E
:10323000FF080020FFF73BFEC4B20020FFF737FE77
:10324000C1B2B56100BF00BF00BF00BF00BF00BF7B
:1032500000BF00BF00BF00BF00BF00BF00BF00BF76
:1032600000BF00BF00BF00BF00BF00BF00BF00BF66
:1032700000BF00BF00BF00BF00BF00BF00BF00BF56
:1032800000BF00BF174D184E184FB8F1C20F01D143
:10329000202C07D0822028602120306078463860BA
:1032A00082200EE70C48142912D0152920D01629A7
:1032B00022D0182923D0C0F800900020FFF718FE74
:1032C000C5F800907846C6F8009038600020F8E60F
:1032D0004FF480110EE0000034010010008009203E
:1032E000A08601006C000010700000107400001037
:1032F0004FF400110160E0E74FF48001FAE74FF06E
:103300008071F7E72DE9F34FC3B0804600244FF0FA
:10331000820AFE4DFE4EFF4F4FF0210BA14641A900
:10332000FD4800F032FA00286AD100F099FA022034
:103330008DF800004FEA18108DF8010004EB08101A
:103340008DF8020044988DF8039000EB04214FF4AF
:10335000807201A8FDF742F800BF00BF00BF00BFA8
:1033600000BF00BF00BF00BF00BF00BF00BF00BF65
:1033700000BF00BF00BF00BF00BF00BF00BF00BF55
:1033800000BF00BF00BF00BF00BF00BF00BF00BF45
:1033900000BF00BF00BF00BF4020E049C8614FF43C
:1033A00082716846FFF78AFDDC494020886100BFD2
:1033B00000BF00BF00BF00BF00BF00BF00BF00BF15
:1033C00000BF00BF00BF00BF00BF00BF00BF00BF05
:1033D00000BF00BF00BF00BF00BF00BF00BF00BFF5
:1033E00000BF00BF00BF00BF00BF00BF00BF641C24
:1033F000E4B2102C93D341A9C74800F0C6F948B1F4
:10340000C5F800A07846C6F800B03860822045B004
:10341000BDE8F08F00F06DFAC5F800907846C6F868
:10342000009038600020F2E72DE9F04F89B0DFF816
:10343000DC825FEA020B4FF0000607910FD04FF4D9
:10344000805501462A466846FCF73EFFDDE9004705
:10345000284602F035F85FEA00090CD016E0862114
:10346000AB48C8F80010092101607946A9480160FD
:10347000862009B0CCE78221A548C8F80010222197
:1034800001607946A34801608220F2E7ABEB0605B4
:10349000C7F580504FF0000AA84200D20546B5F5A6
:1034A000805F04D02046494600F09DFCD8B90798BB
:1034B0002A46811907EB0900FCF790FF204600F02F
:1034C00018FC80B920464946FFF71CFF58B9204632
:1034D0004946FFF7F8FD78B10AF1010000F0FF0A54
:1034E000BAF1030F05D3484601F0C2FFD8F8000037
:1034F000BFE7BAF1000FE1D12E440027641C5E45FE
:10350000C4D3484601F0B4FF81490020C8F8000048
:10351000086079467F4801600020AAE72DE9FF4F47
:103520008DB00D46DDF868900026784C07935FEA71
:1035300009013ED04FF4805701463A466846FCF7F1
:10354000C3FEDDE900B10C913A46691C6846FCF700
:10355000BBFEDDE90010CDE904013A4668460F994B
:10356000FCF7B2FEDDE90085A9EB0607C5F5805042
:10357000B84200D2074625B1D8457CD10C98854287
:1035800079D14FF4805001F09BFF5FEA000A1BD015
:10359000D8454FD10C9885424CD12A464FEA083085
:1035A000514600F0FAFA000618D5504601F060FFC7
:1035B00079E0862020605648092101607846554907
:1035C0000860862011B023E7822020605048222125
:1035D000016079464F4801608220F3E705988045F5
:1035E00009D1049901EB0030C1F58052514400F03B
:1035F000D4FA0006D9D4404600F07BFB0006D4D4B0
:1036000007983A46811905EB0A00FCF7E7FEEA192C
:103610004FEA0830514601F0D3F90006C5D40599A8
:10362000884533D1049800EB01300499C1F58052EC
:10363000514427E0059988450AD1049800EB0130F0
:103640000499C1F58052514600F0A7FA0006ACD4A7
:10365000404600F04EFB0006A7D407983A46811971
:103660000F98304401F0ACF900069ED405998845C6
:103670000CD1049800E00DE000EB01300499C1F595
:103680008052514601F09CF900068ED4504601F05C
:10369000EFFE0AE007983A4681190F98304401F08E
:1036A0008FF9000601D520688CE73E44002508F11B
:1036B00001084E45FFF458AF15490020206008600E
:1036C00078461449086000207CE715480068704778
:1036D0004FF4805070472DE9F04FDFF83080DFF86D
:1036E00030B089B00F0004464FF0000634D04FF4DC
:1036F000805501462A466846FCF7E6FDDDE900A153
:1037000005912A46214606A80CE000006C00001036
:103710007000001074000010A086010000800920D5
:1037200034010010FCF7D0FDDDE906404FF0000940
:10373000BD1BC0F58051A94200D20D4620B15445B1
:1037400015D10599884212D1204600F0D2FA000620
:103750000DD5D8F800008CE68621C8F800100921A4
:10376000CBF8001079463B480160862081E62E4464
:10377000641C4846BE42DBD3C8F800007946CBF84B
:10378000000034480160002073E62DE9F041324C1E
:103790000F460646A56806E0A068401BB04202D36B
:1037A0000120BDE8F081384600F003F80028F3D18D
:1037B000F7E770B5044600BF00BF00BF00BF00BF01
:1037C00000BF00BF00BF00BF00BF00BF00BF00BF01
:1037D00000BF00BF00BF00BF00BF00BF00BF00BFF1
:1037E00000BF00BF00BF00BF00BF00BF00BF00BFE1
:1037F00000BF00BF00BF4025184EF5610520FFF750
:1038000056FB0020FFF753FB2070B56100BF00BFDF
:1038100000BF00BF00BF00BF00BF00BF00BF00BFB0
:1038200000BF00BF00BF00BF00BF00BF00BF00BFA0
:1038300000BF00BF00BF00BF00BF00BF00BF00BF90
:1038400000BF00BF00BF00BF00BF00BF207800F076
:10385000010070BD740000100000094000800920C4
:1038600070B500BF00BF00BF00BF00BF00BF00BFFA
:1038700000BF00BF00BF00BF00BF00BF00BF00BF50
:1038800000BF00BF00BF00BF00BF00BF00BF00BF40
:1038900000BF00BF00BF00BF00BF00BF00BF00BF30
:1038A00000BF4025FB4CE5610620FFF700FBA5614A
:1038B00000BF00BF00BF00BF00BF00BF00BF00BF10
:1038C00000BF00BF00BF00BF00BF00BF00BF00BF00
:1038D00000BF00BF00BF00BF00BF00BF00BF00BFF0
:1038E00000BF00BF00BF00BF00BF00BF00BF00BFE0
:1038F00070BD70B500BF00BF00BF00BF00BF00BFFC
:1039000000BF00BF00BF00BF00BF00BF00BF00BFBF
:1039100000BF00BF00BF00BF00BF00BF00BF00BFAF
:1039200000BF00BF00BF00BF00BF00BF00BF00BF9F
:1039300000BF00BF4025D74CE5610420FFF7B7FA70
:10394000A56100BF00BF00BF00BF00BF00BF00BF38
:1039500000BF00BF00BF00BF00BF00BF00BF00BF6F
:1039600000BF00BF00BF00BF00BF00BF00BF00BF5F
:1039700000BF00BF00BF00BF00BF00BF00BF00BF4F
:1039800000BF70BD70B5064600BF00BF00BF00BFDE
:1039900000BF00BF00BF00BF00BF00BF00BF00BF2F
:1039A00000BF00BF00BF00BF00BF00BF00BF00BF1F
:1039B00000BF00BF00BF00BF00BF00BF00BF00BF0F
:1039C00000BF00BF00BF00BF4024B24DEC615020DB
:1039D000FFF76DFAAC6100BF00BF00BF00BF00BFC2
:1039E00000BF00BF00BF00BF00BF00BF00BF00BFDF
:1039F00000BF00BF00BF00BF00BF00BF00BF00BFCF
:103A000000BF00BF00BF00BF00BF00BF00BF00BFBE
:103A100000BF00BF00BF00BF00BF00BF00BF00BFAE
:103A200000BF00BF00BF00BF00BF00BF00BF00BF9E
:103A300000BF00BF00BF00BF00BF00BF00BF00BF8E
:103A400000BF00BF00BF00BF00BF00BF00BF00BF7E
:103A500000BF00BF00BFEC610120FFF728FAB000F3
:103A6000FFF725FAAC6100BF00BF00BF00BF00BF79
:103A700000BF00BF00BF00BF00BF00BF00BF00BF4E
:103A800000BF00BF00BF00BF00BF00BF00BF00BF3E
:103A900000BF00BF00BF00BF00BF00BF00BF00BF2E
:103AA00000BF00BF00BF70BD2DE9FE430F460446B6
:103AB00002A9794800F0B8FD784D794EDFF8E4812D
:103AC00048B1822028602220794630608220C8F8E0
:103AD0000010BDE8FE839DF80800800701D4FFF7C1
:103AE000BFFE02208DF80000200C8DF80100200A96
:103AF0008DF802008DF803408DF8047000BF00BF00
:103B000000BF00BF00BF00BF00BF00BF00BF00BFBD
:103B100000BF00BF00BF00BF00BF00BF00BF00BFAD
:103B200000BF00BF00BF00BF00BF00BF00BF00BF9D
:103B300000BF00BF00BF00BF00BF00BF4024554F03
:103B4000FC6105216846FFF7B9F9BC6100BF00BF01
:103B500000BF00BF00BF00BF00BF00BF00BF00BF6D
:103B600000BF00BF00BF00BF00BF00BF00BF00BF5D
:103B700000BF00BF00BF00BF00BF00BF00BF00BF4D
:103B800000BF00BF00BF00BF00BF00BF0020286013
:103B900079463060C8F800109BE72DE9FC5F3F4D87
:103BA0003F4E404F5FEA020A8B4604464FF0000842
:103BB0000DD001A9384800F037FD80B1822028607F
:103BC00021203060784638608220BDE8FC9FC5F82F
:103BD00000807846C6F8008038600020F5E70320B2
:103BE0008DF80000200C8DF80100200A8DF80200ED
:103BF0008DF8034000BF00BF00BF00BF00BF00BF83
:103C000000BF00BF00BF00BF00BF00BF00BF00BFBC
:103C100000BF00BF00BF00BF00BF00BF00BF00BFAC
:103C200000BF00BF00BF00BF00BF00BF00BF00BF9C
:103C300000BF00BF174C4FF04009C4F81C9004218E
:103C40006846FFF73BF951465846FFF742F9C4F87A
:103C5000189000BF00BF00BF00BF00BF00BF00BF83
:103C600000BF00BF00BF00BF00BF00BF00BF00BF5C
:103C700000BF00BF00BF00BF00BF00BF00BF00BF4C
:103C800000BF00BF00BF00BF00BF00BF00BF00BF3C
:103C900000BF9CE700800920A08601006C00001096
:103CA00070000010740000102DE9F05FFE4EDFF888
:103CB000FC93DFF8FCA3150083460F464FF0000885
:103CC0000ED000240AE0395D0BEB0400FFF7ECFE98
:103CD000000602D53068BDE8F09F641CAC42F2D308
:103CE000C6F800807946C9F800800020CAF80010A4
:103CF000F1E72DE9FC47044601A9EE4800F094FCE9
:103D0000E94DEA4EDFF8A89348B1822028602220CE
:103D1000794630608220C9F80010BDE8FC879DF824
:103D20000400800701D4FFF79BFD20208DF80000E0
:103D300020098DF8010020018DF8020000248DF883
:103D4000034000BF00BF00BF00BF00BF00BF00BFF7
:103D500000BF00BF00BF00BF00BF00BF00BF00BF6B
:103D600000BF00BF00BF00BF00BF00BF00BF00BF5B
:103D700000BF00BF00BF00BF00BF00BF00BF00BF4B
:103D800000BF4027DFF83083C8F81C700421684664
:103D9000FFF794F8C8F8187000BF00BF00BF00BF5D
:103DA00000BF00BF00BF00BF00BF00BF00BF00BF1B
:103DB00000BF00BF00BF00BF00BF00BF00BF00BF0B
:103DC00000BF00BF00BF00BF00BF00BF00BF00BFFB
:103DD00000BF00BF00BF00BF2C60794634600020E8
:103DE000C9F8001099E72DE9FC478A46044601A965
:103DF000B04800F019FCAC4DAC4EDFF8B49240B1C5
:103E0000822028602220794630608220C9F8001084
:103E100083E703208DF8000020098DF801002001C0
:103E20008DF8020000248DF8034000BF00BF00BFE2
:103E300000BF00BF00BF00BF00BF00BF00BF00BF8A
:103E400000BF00BF00BF00BF00BF00BF00BF00BF7A
:103E500000BF00BF00BF00BF00BF00BF00BF00BF6A
:103E600000BF00BF00BF00BF00BF4027DFF848828F
:103E7000C8F81C7004216846FFF720F8B9015046C5
:103E8000FFF727F8C8F8187000BF00BF00BF00BFD9
:103E900000BF00BF00BF00BF00BF00BF00BF00BF2A
:103EA00000BF00BF00BF00BF00BF00BF00BF00BF1A
:103EB00000BF00BF00BF00BF00BF00BF00BF00BF0A
:103EC00000BF00BF00BF00BF2C60794634600020F7
:103ED000C9F8001021E72DE9F34F83B0044601A98A
:103EE000744800F0A1FB704D704E714F4FF0820886
:103EF00018B12120C5F800806CE09DF8040080070F
:103F000001D4FFF7ADFCAD208DF8000020098DF83D
:103F1000010020018DF802004FF0000B8DF803B076
:103F200000BF00BF00BF00BF00BF00BF00BF00BF99
:103F300000BF00BF00BF00BF00BF00BF00BF00BF89
:103F400000BF00BF00BF00BF00BF00BF00BF00BF79
:103F500000BF00BF00BF00BF00BF00BF00BF00BF69
:103F6000DFF854914FF0400A5446C9F81CA00421D0
:103F70006846FEF7A3FF02210498FEF79FFFC9F8E9
:103F8000184000BF00BF00BF00BF00BF00BF00BFA0
:103F900000BF00BF00BF00BF00BF00BF00BF00BF29
:103FA00000BF00BF00BF00BF00BF00BF00BF00BF19
:103FB00000BF00BF00BF00BF00BF00BF00BF00BF09
:103FC00000BF022401A93B4800F02EFB48B122208B
:103FD000C5F80080306078463860822005B0BDE8C2
:103FE000F08F00BF00BF00BF00BF00BF00BF00BF19
:103FF00000BF00BF00BF00BF00BF00BF00BF00BFC9
:1040000000BF00BF00BF00BF00BF00BF00BF00BFB8
:1040100000BF00BF00BF00BF00BF00BF00BF00BFA8
:1040200000BFC9F81CA0AD20FEF741FF0498022193
:104030002044FEF743FFC9F818A000BF00BF00BF2F
:1040400000BF00BF00BF00BF00BF00BF00BF00BF78
:1040500000BF00BF00BF00BF00BF00BF00BF00BF68
:1040600000BF00BF00BF00BF00BF00BF00BF00BF58
:1040700000BF00BF00BF00BF00BFA41CA4B2B4F5C6
:10408000805F9FD301A90B4800F0CEFA00287FF48F
:1040900030AFFFF72EFCC5F800B07846C6F800B088
:1040A000386000209AE700006C00001070000010DB
:1040B00074000010A08601000080092070B5FD4D3D
:1040C000FD4EFE4C2AB1FFF768FD000609D52068B9
:1040D00070BD8620206009202860784630608620E8
:1040E00070BD00202060286078463060002070BDE0
:1040F0002DE9F04F89B0DFF8C483DFF8B8B35FEA89
:1041000002094FF0000607910FD04FF48055014689
:104110002A466846FCF7D8F8DDE90047284601F052
:10412000CFF95FEA000A0CD016E08621C8F800102B
:104130000921CBF800107946DF480160862009B0DC
:104140004DE78221C8F800102221CBF800107946F3
:10415000D94801608220F2E7A9EB0605C7F5805037
:10416000A84200D20546B5F5805F04D020465146EE
:10417000FFF739FE80B92046FFF7BBFD60B907980D
:104180002A46811907EB0A00FCF728F92E4420463D
:104190005146FFF7A0FE28B1504601F069F9D8F862
:1041A0000000CCE70027641C4E45D5D3504601F0F3
:1041B0005FF90020C8F800007946CBF80000BE483F
:1041C00001600020BBE72DE9FF4F8DB00D46DDF803
:1041D00068900026B94C07935FEA09013FD04FF47D
:1041E000805701463A466846FCF76EF8DDE900B1B3
:1041F0000C913A46691C6846FCF766F8DDE9001048
:10420000CDE904013A4668460F99FCF75DF8DDE90F
:10421000008500BFA9EB0607C5F58050B84200D263
:10422000074625B1D8457CD10C98854279D14FF409
:10423000805001F045F95FEA000A1BD0D8454FD104
:104240000C9885424CD12A464FEA08305146FFF778
:10425000A4FC000618D5504601F00AF979E0862042
:1042600020609448092101607846934908608620BF
:1042700011B0B4E6822020608E4822210160794688
:104280008D4801608220F3E70598804509D10499A3
:1042900001EB0030C1F580525144FFF77EFC00066F
:1042A000D9D44046FFF725FD0006D4D407983A46F6
:1042B000811905EB0A00FCF791F8EA194FEA08307A
:1042C0005146FFF7F1FC0006C5D40599884533D166
:1042D000049800EB01300499C1F58052514427E065
:1042E000059988450AD1049800EB01300499C1F57D
:1042F00080525146FFF751FC0006ACD44046FFF710
:10430000F8FC0006A7D407983A4681190F98304464
:10431000FFF7CAFC00069ED4059988450CD1049885
:1043200000E00DE000EB01300499C1F580525146E8
:10433000FFF7BAFC00068ED4504601F099F80AE067
:1043400007983A4681190F983044FFF7ADFC0006F4
:1043500001D520688CE73E44002508F101084E4550
:10436000FFF458AF53490020206008607846524956
:10437000086000207CE72DE9F0474FF0000900BFFE
:1043800000BF00BF00BF00BF00BF00BF00BF00BF35
:1043900000BF00BF00BF00BF00BF00BF00BF00BF25
:1043A00000BF00BF00BF00BF00BF00BF00BF00BF15
:1043B00000BF00BF00BF00BF00BF00BF00BF40255F
:1043C0003F4EF5619F20FEF772FD0020FEF76FFD66
:1043D00000F0FF080020FEF76AFDC4B20020FEF7DF
:1043E00066FDC1B2B56100BF00BF00BF00BF00BF26
:1043F00000BF00BF00BF00BF00BF00BF00BF00BFC5
:1044000000BF00BF00BF00BF00BF00BF00BF00BFB4
:1044100000BF00BF00BF00BF00BF00BF00BF00BFA4
:1044200000BF00BF00BF254D224E234FB8F1BF0F84
:1044300003D1252C0AD0262C08D0822028602120E8
:104440003060784638608220BDE8F0871D484129F9
:1044500012D04FF48002422912D04A2910D0C0F85D
:1044600000900020FFF78EFAC5F800907846C6F855
:10447000009038600020E7E74FF400110160F0E79A
:104480000260EEE72DE9F84F69460F4800F0CCF8DE
:1044900082270A4C074D084E4FF0220A002862D1AD
:1044A0009DF80000800701D4FFF7DAF900BF00BFD4
:1044B00000BF0BE070000010740000106C000010D2
:1044C0000080092038010010A086010000BF00BF55
:1044D00000BF00BF00BF00BF00BF00BF00BF00BFE4
:1044E00000BF00BF00BF00BF00BF00BF00BF00BFD4
:1044F00000BF00BF00BF00BF00BF00BF00BF00BFC4
:1045000000BF00BF00BFDFF8EC914FF04008C9F8D2
:104510001C806020FEF7CBFCC9F8188000BF00BFEC
:1045200000BF00BF00BF00BF00BF00BF00BF00BF93
:1045300000BF00BF00BF00BF00BF00BF00BF00BF83
:1045400000BF00BF00BF00BF00BF00BF00BF00BF73
:1045500000BF00BF00BF00BF00BF00BF6946664884
:1045600000F062F838B127607846C5F800A03060E6
:104570008220BDE8F88F00202060286078463060F7
:104580000020F6E75D48006870474FF480507047A0
:104590002DE9F04FDFF86881DFF868B189B00F00CE
:1045A00004464FF0000626D04FF4805501462A46B7
:1045B0006846FBF789FEDDE900A105912A46214600
:1045C00006A8FBF781FEDDE906404FF00009BD1BA0
:1045D000C0F58051A94200D20D4620B1544515D1F5
:1045E0000599884212D12046FFF783FB00060DD5BE
:1045F000D8F80000A3E58621C8F800100921CBF8FF
:104600000010794640480160862098E52E44641CDD
:104610004846BE42DBD3C8F800007946CBF800001C
:104620003948016000208AE52DE9F041374C0F46FA
:104630000646A56806E0A068401BB04202D30120F0
:10464000BDE8F081384600F003F80028F3D1F7E721
:1046500070B5044600BF00BF00BF00BF00BF00BF71
:1046600000BF00BF00BF00BF00BF00BF00BF00BF52
:1046700000BF00BF00BF00BF00BF00BF00BF00BF42
:1046800000BF00BF00BF00BF00BF00BF00BF00BF32
:1046900000BF00BF4025174EF5610520FEF707FC5F
:1046A0000020FEF704FC2070B56100BF00BF00BF12
:1046B00000BF00BF00BF00BF00BF00BF00BF00BF02
:1046C00000BF00BF00BF00BF00BF00BF00BF00BFF2
:1046D00000BF00BF00BF00BF00BF00BF00BF00BFE2
:1046E00000BF00BF00BF00BF00BF207800F0010086
:1046F00070BD00000080092020A1070038010010D3
:104700006C000010700000107400001000000940E0
:104710002DE9FF4703A9FE4800F05FFBFD4DFE4E6B
:10472000DFF8F89350B1822028602120794630606C
:104730008220C9F8001004B0BDE8F0879DF80C0095
:10474000800701D4FFF78CF842208DF80000002488
:10475000CDF80140CDF80540ADF8094000BF00BFDD
:1047600000BF00BF00BF00BF00BF00BF00BF00BF51
:1047700000BF00BF00BF00BF00BF00BF00BF00BF41
:1047800000BF00BF00BF00BF00BF00BF00BF00BF31
:1047900000BF00BF00BF00BF00BF00BF4027DFF861
:1047A0008083C8F81C700B216846FEF787FBC8F8A9
:1047B000187000BF00BF00BF00BF00BF00BF00BF38
:1047C00000BF00BF00BF00BF00BF00BF00BF00BFF1
:1047D00000BF00BF00BF00BF00BF00BF00BF00BFE1
:1047E00000BF00BF00BF00BF00BF00BF00BF00BFD1
:1047F00000BF2C60794634600020C9F800109AE7A9
:104800002DE9F34F85B0044603A9C14800F0E5FA4D
:10481000C04DC14EC14F4FF0820B18B12120C5F8D9
:1048200000B060E0FFF71CF842208DF800004FF068
:10483000000ACDF801A0CDF805A0ADF809A000BF91
:1048400000BF00BF00BF00BF00BF00BF00BF00BF70
:1048500000BF00BF00BF00BF00BF00BF00BF00BF60
:1048600000BF00BF00BF00BF00BF00BF00BF00BF50
:1048700000BF00BF00BF00BF00BF00BF00BFDFF828
:10488000A0924FF04008C9F81C800B216846FEF743
:1048900015FBC9F8188000BF00BF00BF00BF00BFF4
:1048A00000BF00BF00BF00BF00BF00BF00BF00BF10
:1048B00000BF00BF00BF00BF00BF00BF00BF00BF00
:1048C00000BF00BF00BF00BF00BF00BF00BF00BFF0
:1048D00000BF00BF00BF03A98D4800F07EFA48B1B9
:1048E0002220C5F800B0306078463860822007B0DA
:1048F000BDE8F08F9DF80C00800701D4FEF7B0FFF3
:1049000002208DF80000200C8DF80100200A8DF89F
:10491000020006988DF803408DF8040000BF00BF28
:1049200000BF00BF00BF00BF00BF00BF00BF00BF8F
:1049300000BF00BF00BF00BF00BF00BF00BF00BF7F
:1049400000BF00BF00BF00BF00BF00BF00BF00BF6F
:1049500000BF00BF00BF00BF00BF00BF4446C84645
:10496000C9F81C4005216846FEF7A8FAC8F81840A7
:1049700000BF00BF00BF00BF00BF00BF00BF00BF3F
:1049800000BF00BF00BF00BF00BF00BF00BF00BF2F
:1049900000BF00BF00BF00BF00BF00BF00BF00BF1F
:1049A00000BF00BF00BF00BF00BF00BF00BF00BF0F
:1049B000C5F800A07846C6F800A03860002096E749
:1049C0002DE9F05F534EDFF85091DFF850A115004C
:1049D00083460F464FF000080ED000240AE0395DF0
:1049E0000BEB0400FFF70CFF000602D53068BDE8B2
:1049F000F09F641CAC42F2D3C6F800807946C9F837
:104A000000800020CAF80010F1E72DE9F34F0024E0
:104A1000404D414E414FC3B080464FF0820A4FF0A7
:104A2000210BA14641A93A4800F0D7F900286ED1E0
:104A30009DF80401800701D4FEF712FF02208DF8D3
:104A400000004FEA18108DF8010004EB08108DF8F3
:104A5000020044988DF8039000EB04214FF480721B
:104A600001A8FBF7BBFC00BF00BF00BF00BF00BF39
:104A700000BF00BF00BF00BF00BF00BF00BF00BF3E
:104A800000BF00BF00BF00BF00BF00BF00BF00BF2E
:104A900000BF00BF00BF00BF00BF00BF00BF00BF1E
:104AA00000BF00BF00BF40201D49C8614FF48271A4
:104AB0006846FEF703FA1A494020886100BF00BF2C
:104AC00000BF00BF00BF00BF00BF00BF00BF00BFEE
:104AD00000BF00BF00BF00BF00BF00BF00BF00BFDE
:104AE00000BF00BF00BF00BF00BF00BF00BF00BFCE
:104AF00000BF00BF00BF00BF00BF00BF641CE4B226
:104B0000102C8FD341A9024800F067F998B109E051
:104B1000A08601006C0000107000001074000010EE
:104B200000800920C5F800A07846C6F800B03860BB
:104B3000822045B0DCE6FEF7DCFEC5F80090784642
:104B4000C6F8009038600020F3E72DE9F04F89B0F7
:104B5000DFF85083DFF850B35FEA02094FF0000638
:104B600007910FD04FF4805501462A466846FBF75F
:104B7000ABFBDDE90047284600F0A2FC5FEA000A33
:104B80000CD016E08621C8F800100921CBF80010DF
:104B90007946C6480160862009B0A9E68221C8F896
:104BA00000102221CBF800107946C0480160822015
:104BB000F2E7A9EB0605C7F58050A84200D20546EA
:104BC000B5F5805F04D020465146FFF70CF980B957
:104BD0002046FFF78EF860B907982A46811907EB3F
:104BE0000A00FBF7FBFB2E4420465146FFF70DFF62
:104BF00028B1504600F03CFCD8F80000CCE7002774
:104C0000641C4E45D5D3504600F032FC0020C8F855
:104C100000007946CBF80000A44801600020BBE703
:104C20002DE9FF4F8DB00D46DDF8689000269D4CB4
:104C300007935FEA09013ED04FF4805701463A4698
:104C40006846FBF741FBDDE900B10C913A46691C6F
:104C50006846FBF739FBDDE90010CDE904013A466F
:104C600068460F99FBF730FBDDE90085A9EB0607E5
:104C7000C5F58050B84200D2074625B1D8457CD151
:104C80000C98854279D14FF4805000F019FC5FEA0E
:104C9000000A1BD0D8454FD10C9885424CD12A46EA
:104CA0004FEA08305146FEF778FF000618D5504607
:104CB00000F0DEFB79E0862020607B48092101605E
:104CC00078467A490860862011B011E6822020607B
:104CD0007548222101607946744801608220F3E71B
:104CE0000598804509D1049901EB0030C1F5805247
:104CF0005144FEF752FF0006D9D44046FEF7F9FFB3
:104D00000006D4D407983A46811905EB0A00FBF750
:104D100065FBEA194FEA08305146FFF751FE0006DD
:104D2000C5D40599884533D1049800EB0130049926
:104D3000C1F58052514427E0059988450AD104986D
:104D400000EB01300499C1F580525146FEF725FF72
:104D50000006ACD44046FEF7CCFF0006A7D4079867
:104D60003A4681190F983044FFF72AFE00069ED478
:104D7000059988450CD1049800E00DE000EB013066
:104D80000499C1F580525146FFF71AFE00068ED4F1
:104D9000504600F06DFB0AE007983A4681190F98DB
:104DA0003044FFF70DFE000601D520688CE73E4435
:104DB000002508F101084E45FFF458AF3A4900209C
:104DC0002060086078463949086000207CE74FF48D
:104DD000800070474FF4805070472DE9F041344C0B
:104DE0000F460646A56806E0A068401BB04202D305
:104DF0000120BDE8F081384600F003F80028F3D127
:104E0000F7E770B5044600BF00BF00BF00BF00BF9A
:104E100000BF00BF00BF00BF00BF00BF00BF00BF9A
:104E200000BF00BF00BF00BF00BF00BF00BF00BF8A
:104E300000BF00BF00BF00BF00BF00BF00BF00BF7A
:104E400000BF00BF00BF40251A4EF5610520FEF7E8
:104E50002EF80020FEF72BF82070B56100BF00BFD0
:104E600000BF00BF00BF00BF00BF00BF00BF00BF4A
:104E700000BF00BF00BF00BF00BF00BF00BF00BF3A
:104E800000BF00BF00BF00BF00BF00BF00BF00BF2A
:104E900000BF00BF00BF00BF00BF00BF207800F010
:104EA000010070BD6C000010700000107400001054
:104EB000000009400080092000207047AE49822090
:104EC0000860AE49212008607846AD49086082201C
:104ED0007047A94982200860A849222008607846C6
:104EE000A749086082207047A34982200860A3492F
:104EF000222008607846A24908608220704770B579
:104F0000002400BF00BF00BF00BF00BF00BF00BF44
:104F100000BF00BF00BF00BF00BF00BF00BF00BF99
:104F200000BF00BF00BF00BF00BF00BF00BF00BF89
:104F300000BF00BF00BF00BF00BF00BF00BF00BF79
:104F400000BF40258F4EF5619F20FDF7B0FF002088
:104F5000FDF7ADFF60F307040020FDF7A8FF60F345
:104F60000F240020FDF7A3FF60F31744B56100BFD5
:104F700000BF00BF00BF00BF00BF00BF00BF00BF39
:104F800000BF00BF00BF00BF00BF00BF00BF00BF29
:104F900000BF00BF00BF00BF00BF00BF00BF00BF19
:104FA00000BF00BF00BF00BF00BF00BF00BF764909
:104FB000601A8C421AD00BDCA4F1C204B4F5A1141F
:104FC00014D0B4F5803F11D0B4F5003F0BD10DE003
:104FD0006E49401805D06E49401809D06D49C84245
:104FE00001D1022400E00024204670BD0324FBE729
:104FF0000424FFF78DFBF7E76748007828B167497D
:1050000000EBC00051F8200000475B498220086097
:105010005A49212008607846594908608220704723
:1050200070B5FFF76CFF5C49544D554E524C0870FB
:1050300050B15A4900EBC00001EB80008068804706
:10504000000609D5206870BD8220206021202860DC
:1050500078463060822070BD00202060286078464D
:105060003060002070BD2DE9F0414B4B434D444E64
:105070001B78414C63B19AB1484F03EBC30307EB74
:1050800083031B699847000612D52068BDE8F081AC
:105090008220206021202860784630608220F5E759
:1050A0008620206009202860784630608620EDE761
:1050B000002020602860784630600020E6E72DE977
:1050C000F041354B2D4D2E4E1B782B4C5BB192B1E0
:1050D000324F03EBC30307EB83039B69984700063A
:1050E00011D52068D2E782202060222028607846EF
:1050F00030608220CAE78620206009202860784638
:1051000030608620C2E7002020602860784630604A
:105110000020BBE7F8B5204C184D194E2778164CE7
:10512000DDF818C087B1BCF1000F15D0CDF800C074
:10513000DFF868C007EBC7070CEB8707FF69B847C4
:10514000000611D52068F8BD82202060222028604A
:10515000784630608220F8BD8620206009202860D3
:10516000784630608620F8BD0020206028607846B0
:1051700030600020F8BD00006C00001070000010CE
:105180007400001000800920C220180003FBD6FF25
:1051900000FFFEFF0001F8FF3C010010405C000032
:1051A000D2B201E000F8012B491EFBD27047002269
:1051B000F6E710B513460A4604461946FFF7F0FF16
:1051C000204610BD30B50B460146002020220124A8
:1051D00009E021FA02F59D4205D303FA02F5491BC5
:1051E00004FA02F52844151EA2F10102F1DC30BDDB
:1051F00070B500242546002801DA01244042002928
:1052000001DA01254942FFF7DDFFAC4200D0404200
:10521000002C00D0494270BD064C074D06E0E06806
:1052200040F0010394E8070098471034AC42F6D3ED
:10523000FAF75CFF185D0000485D000030B58C187F
:1052400010F8012B12F00F0301D110F8013B1209E5
:1052500006D110F8012B03E010F8015B01F8015BA7
:105260005B1EF9D101E001F8013B521EFBD1A142C6
:10527000E6D3002030BD00000FB41CB50A46521E14
:10528000CDE9000207A9054B6A46069800F008F828
:10529000009A002111701CBC5DF814FB59540000E9
:1052A0002DE9FF4F8BB09A460F460546002606E0D3
:1052B00025280BD052460D9990476D1C761C2878F6
:1052C0000028F5D10FB03046BDE8F08F0024A0468D
:1052D0000122604900E0044315F8013F203B02FA37
:1052E00003F00842F7D128782E2817D115F8010FBE
:1052F00044F004042A280ED06FF02F022878A0F181
:10530000300109290AD808EB880102EB410100EBC2
:1053100001086D1CF2E757F8048B6D1C287869288A
:105320003ED006DC0028CDD063280BD0642804D101
:1053300036E0732810D075284BD052460D9990470F
:10534000761C85E017F8040B8DF8000000208DF81E
:105350000100E946012003E057F8049B4FF0FF30BD
:1053600061074FF0000401D40AE0641C44450DDAE3
:105370008442FADB19F804100029F6D106E0641C17
:105380008442FCDB19F804100029F8D1264404E01B
:1053900019F8010B52460D999047641EF8D257E058
:1053A00001CF4FF00A0B002802DA40422D2102E023
:1053B000210504D52B218DF82410012103E0E107FC
:1053C00005D02021F7E70DF1200908910CE000211C
:1053D000F9E701CF4FF00A0BF9E75946FFF7F2FE64
:1053E00001F1300209F8012D0028F6D1ADEB0900DA
:1053F00000F1200B600701D44FF00108D84502DD11
:10540000A8EB0B0000E000208046002406E009A87D
:105410005246005D0D999047641C761C08988442A2
:10542000F5DB04E0302052460D999047761CB8F128
:105430000001A8F10108F5DC05E019F8010B52465E
:105440000D999047761CBBF10001ABF1010BF4DC28
:105450006D1C34E7092801004A68002A06D00A6852
:10546000531C0B6010704868401E48607047000075
:1054700010B5002821D0114B0022001F196803E04D
:10548000814203D80A4649680029F9D152B113680C
:10549000841A9C4204D1006818441060104602E04F
:1054A000506000E0186039B102680B1A934203D1D2
:1054B0000B681A4402604968416010BD4001001049
:1054C000F0B50B30154D20F007010024144A0FE011
:1054D00003688B420BD38B4205D95E1A4318476889
:1054E000C3E9006700E04368136002C004E0021DE6
:1054F00010680028ECD12046002802D1286808B1A5
:105500000020F0BD064A07481060074A121A22F030
:105510000702C0E9002401202860D7E744010010F9
:10552000400100108C1D0010888D001000050F0A2E
:105530001B1E141133363C39282D272263666C69F3
:10554000787D777250555F5A4B4E4441C3C6CCC9E3
:10555000D8DDD7D2F0F5FFFAEBEEE4E1A0A5AFAAD3
:10556000BBBEB4B193969C99888D878283868C89C3
:10557000989D9792B0B5BFBAABAEA4A1E0E5EFEAB3
:10558000FBFEF4F1D3D6DCD9C8CDC7C240454F4AA3
:105590005B5E545173767C79686D676223262C2993
:1055A000383D373210151F1A0B0E040103060C0983
:1055B000181D171230353F3A2B2E242160656F6A73
:1055C0007B7E747153565C59484D4742C0C5CFCA63
:1055D000DBDED4D1F3F6FCF9E8EDE7E2A3A6ACA953
:1055E000B8BDB7B290959F9A8B8E848180858F8A43
:1055F0009B9E9491B3B6BCB9A8ADA7A2E3E6ECE933
:10560000F8FDF7F2D0D5DFDACBCEC4C143464C4922
:10561000585D575270757F7A6B6E646120252F2A12
:105620003B3E343113161C19080D070200002110EF
:10563000422063308440A550C660E77008812991FC
:105640004AA16BB18CC1ADD1CEE1EFF131121002A4
:1056500073325222B5529442F772D662399318834C
:105660007BB35AA3BDD39CC3FFF3DEE36224433470
:1056700020040114E664C774A44485546AA54BB59C
:1056800028850995EEE5CFF5ACC58DD55336722644
:1056900011163006D776F6669556B4465BB77AA7EC
:1056A00019973887DFF7FEE79DD7BCC7C448E55890
:1056B0008668A7784008611802282338CCC9EDD93C
:1056C0008EE9AFF9488969990AA92BB9F55AD44AE4
:1056D000B77A966A711A500A333A122AFDDBDCCB8C
:1056E000BFFB9EEB799B588B3BBB1AABA66C877CB0
:1056F000E44CC55C222C033C600C411CAEED8FFDDC
:10570000ECCDCDDD2AAD0BBD688D499D977EB66E83
:10571000D55EF44E133E322E511E700E9FFFBEEF2B
:10572000DDDFFCCF1BBF3AAF599F788F8891A981ED
:10573000CAB1EBA10CD12DC14EF16FE18010A100D7
:10574000C230E3200450254046706760B9839893C7
:10575000FBA3DAB33DC31CD37FE35EF3B102901227
:10576000F322D2323542145277625672EAB5CBA593
:10577000A89589856EF54FE52CD50DC5E234C32477
:10578000A01481046674476424540544DBA7FAB767
:105790009987B8975FE77EF71DC73CD7D326F236C7
:1057A0009106B01657667676154634564CD96DC9B3
:1057B0000EF92FE9C899E9898AB9ABA94458654817
:1057C00006782768C018E1088238A3287DCB5CDB07
:1057D0003FEB1EFBF98BD89BBBAB9ABB754A545A67
:1057E000376A167AF10AD01AB32A923A2EFD0FEDD3
:1057F0006CDD4DCDAABD8BADE89DC98D267C076CB7
:10580000645C454CA23C832CE01CC10C1FEF3EFFA6
:105810005DCF7CDF9BAFBABFD98FF89F176E367E06
:10582000554E745E932EB23ED10EF01E005EBCE269
:10583000613FDD83C29C7E20A3FD1F419DC3217F6C
:10584000FCA2401E5F01E3BD3E6082DC237D9FC160
:10585000421CFEA0E1BF5D0380DE3C62BEE0025C54
:10586000DF81633D7C22C09E1D43A1FF4618FAA440
:1058700027799BC584DA3866E5BB5907DB8567392C
:10588000BAE406581947A5FB7826C49A653BD98720
:10589000045AB8E6A7F91B45C6987A24F8A6441A14
:1058A00099C7257B3A6486D85B05E7B98CD2306E00
:1058B000EDB3510F4E10F2AC2F7193CD114FADF3EC
:1058C000702ECC92D38D6F31B2EC0E50AFF1134DE0
:1058D000CE90722C6D33D18F0C52B0EE326C8ED0D4
:1058E000530DEFB1F0AE4C1291CF2D73CA947628C0
:1058F000ABF517490856B4EA6937D58B5709EBB5AC
:1059000036688AD495CB2977F4AA4816E9B7550B9F
:1059100088D6346A2B7597C94A14F6A8742AC89693
:10592000154BA9F7B6E80A54D7896B35EB3C904D77
:1059300053444F53352E3000020201000110000085
:1059400004F80C000100010000000000000000004D
:10595000000029EFBEADDE41544F4C204650726925
:105960006E744641543132202020000000000000B7
:105970000010000000200000003000000040000087
:105980000050000000600000007000000080000077
:105990000090000000A0000000B0000000C0000067
:1059A00000D0000000E0000000F000000000010056
:1059B00000800100000002000080020000000300DF
:1059C00000800300000004000080040000000500C7
:1059D00000800500000006000080060000000700AF
:1059E00000800700FF0F0000FF1F0000FF2F0000D6
:1059F000FF3F0000FF4F0000FF5F0000FF6F00004F
:105A0000FF7F0000FF8F0000FF9F0000FFAF00003E
:105A1000FFBF0000FFCF0000FFDF0000FFEF00002E
:105A2000FFFF0000FF7F0100FFFF0100FF7F02007A
:105A3000FFFF0200FF7F0300FFFF0300FF7F040062
:105A4000FFFF0400FF7F0500FFFF0500FF7F06004A
:105A5000FFFF0600FF7F0700FFFF0700A11B0000FC
:105A6000A11B0000CF1E0000A11B0000A11B000015
:105A7000A11B0000A11B0000A11B0000A11B000036
:105A8000A11B0000A11B0000A11B0000A11B000026
:105A9000A11B0000A11B0000A11B0000A31B000014
:105AA000A31B0000F9200000A31B0000A31B0000A3
:105AB000A31B0000A31B0000A31B0000A31B0000EE
:105AC000A31B0000A31B0000A31B0000A31B0000DE
:105AD000A31B0000A31B0000A31B0000A51B0000CC
:105AE000A51B0000A91B0000A51B0000A51B0000B2
:105AF000A51B0000A51B0000A51B0000A51B0000A6
:105B0000A51B0000A51B0000A51B0000A51B000095
:105B1000A51B0000A51B0000A51B0000A71B000083
:105B2000A71B0000A71B0000A71B0000A71B00006D
:105B3000A71B0000A71B0000A71B0000A71B00005D
:105B4000A71B0000A71B0000A71B0000A71B00004D
:105B5000A71B0000A71B0000A71B000012011001DB
:105B60000000004051C20313000104204801090253
:105B70002000010100803209040000020806506282
:105B800007058202400000070502024000000004F1
:105B90000309041C03410054004F004C0020002066
:105BA00000200020002000200020002000200028ED
:105BB0000346005000720069006E00740020004629
:105BC000006C0061007300680020002000200020AD
:105BD000002000200020001A034600690072006DBA
:105BE0000077006100720065003000300030003046
:105BF000000E034D0065006D006F0072007900001B
:105C0000CD28000000000000632E0000000000000E
:105C10000000000000000000000000000000000084
:105C20000000000000000000000000000000000074
:105C30000000000000000000000000000000000064
:105C4000B94E0000B94E0000BD4E0000D34E00001A
:105C5000BD4E0000D34E0000D34E0000D34E0000D6
:105C6000E94E0000B94E0000B94E0000BD4E0000E4
:105C7000D34E0000BD4E0000D34E0000D34E0000B6
:105C8000D34E0000E94E0000854500008B45000022
:105C90007743000085440000BD400000F140000053
:105CA000A93C0000C741000091450000CB36000030
:105CB000D1360000D531000085440000BD40000011
:105CC00029340000C14900001D350000D73600000E
:105CD000CF4D0000D54D0000774300008544000003
:105CE000BD4000004B4B0000C1490000214C0000AA
:105CF00091450000000000000000000000000000CE
:105D00000000000000000000000000000000000093
:105D10000000000000000000485D000000000010CE
:105D2000480100003C520000705D00004801001076
:105D3000408C0000EC020000705D000000000020BC
:105D400000100000EC020000BD41544F4C204650B2
:105D500072696E7428054AD4284B3D0286102C0EB9
:105D6000270780C3C9010087930305506CDC02013B
:105D700059855AE4BE15347F33E37FCF673AD0901C
:105D800086F49920329593935C16958201F8626AA5
:105D90000D510D895B51240703E61B48E17FA4DC0C
:105DA000C36CCF3399D975F49F6AFFB5D7140189B5
:105DB0002335C8357533C9F784EF258B215EFCB2D6
:105DC00021FAC18E3EDFCA3D5C58E440572D60F495
:105DD00086064F37BD8A3EAB791F58B56A73524964
:105DE0001EB23BE9A521667862767C08948D88B660
:105DF0003C3D8F110BF80C50AB78F19CB0CBDB5BCA
:105E0000BA4368007DBC439E5AC7B7021A38B4042F
:105E1000DD62501EC91D3BED35DAC12D7C3EFE2CE6
:105E20003F81E491A208673993354D02F0FE63C5C6
:105E3000E2555791C693B026039B57B222D500FF77
:105E4000F08D13C371AEEDA4FBBEF276D1CBE2812F
:105E50009D7B8D517AE014FF2D9AF54AFFEC672B5C
:105E60002CED85063EC298C11B50FF20F3A83E1CB6
:105E7000E2858FE3AE776DE15B7976714D433656FF
:105E8000147CF783BA187419085BADFCA2D163497E
:105E90006008A9347BFAEF3B2DE150A554187B3004
:105EA00014073C2639E651E7561E12894066DA4C43
:105EB0000B4E7FE8CD829C5E19A45B1AA45AF510A4
:105EC0004B0DFCAC276DCD9ACE1C47750947096573
:105ED0005FB43FB35D766B1AED1BC6192749B49DBD
:105EE00091065AB013CA7DBBA9E2B4A8E93FA7093D
:105EF000726FAC405EDE787679801087670E00AEF8
:105F0000644C52DE5892FD66F89E6B08F65130984C
:105F1000BD0D186AA4C7B950A7FB83C4978CC704EA
:105F2000D15AC681C52259E34650024F27502C97BB
:105F300088E5657C513D4E01A3FE86C65F8FB86F34
:105F400024F89B6AACABCE738D15E5593377EB9F84
:105F5000BE68F160CB8390D9184205B05F676200DC
:105F60008CDC5D805B8C8ED2A908286CDD37BC6828
:105F700096A629E7383986B5D6176BF82788D55AFB
:105F80002735E1F579D8DAD254112FC3919A7038B8
:105F9000CB79836D0D432C3BF9793410962C3D0859
:105FA000780DC244CCD3F0E3578A76AB11A1FFC47D
:105FB000B7AA0A77C7216C420B9F197263C34EE4DC
:105FC00049914EE9354841050C3EC37D24D853E242
:105FD000D3D5BE75DA68B7F6D740C49F5941E04DB6
:105FE0005C38AE64B69A86259FFF5765E975AE0AA0
:105FF00027F8109EAED96622F0D361D62CA7B677CB
:00000001FF
